:20400000800F00000000801302EF048021018031018048547765616B5449208081018090A2
:2040200003260904046F1B80020D40A16B99F659BC67F5859C096C0FB4039BC903322CE0E0
:204040000320E32CF42D73B427C4A07254B9EA7C3BAA16F677837AEE1AD4424C6B8B131F7F
:20406000BB938BFC191C3CEC4DE575807F0000000000000000000000000000000000000068
:20408000218D40DB06EFE44FCD5000274083B728177811070021AA401910FD115A8401077A
:2040A00000EDB0AF215A84C93CC901020304050607000016090912120000111111130E002B
:2040C0000011110A0A040000111115150A0010181E181000041F0E0E0E000000000E0E0E6B
:2040E0001F040205040404140800110A040A11000000000E0A0E00000000040E04000000F8
:204100000000040000000000001C0808060106010600001F18181E18181807040404140C73
:204120000402021A020200000C0204080E00000000010204081F0C12120C00000016181089
:20414000100000000E0404040400000106180601001F02021F041F0808100C030C1000005B
:204160000000070000000000000F080E080F0004021F02040000000E191F1919040E15042E
:2041800004040404040404150E0400000000000000040404040004040A0A0A000000000A9C
:2041A0000A1F0A1F0A0A0A0A0E02020000181902040813030814140815120D0404040000A6
:2041C000000002040808080402080402020204080004150E1504000004041F04040000002E
:2041E00000000C04080000001F00000000000000000C0C000102040810000E1113151911E0
:204200000E040C040404040E0E11010204081F1F02040201110E1212121F0202021F101E26
:204220000101110E0608101E11110E1F0102040808080E11110E11110E0E11110F01020CF7
:20424000000C0C000C0C00000C0C000C04080204081008040200001F001F00000804020185
:204260000204080E1101020400040E11151714100F00000D1212120D00001F1111111100D5
:2042800000111111110E000004040A111F000010080F08100008040206091100001F1010DE
:2042A0001010000011111111110000110E1F0E110000010101011E000012141814120000A6
:2042C000040404040400000E111111110000090B0D0101000006091F0906000E11110E01D9
:2042E0000100040E15150E04000001011F10101E01010E10100F00001F1111111F00000E52
:204300001115110E0000040A0A11110000150E0404040000110A040A11000015150E0E046B
:2043200000000000040A1F0609111F11120C001008040201000C04040404040C040A110078
:204340000000000000000000001F0404020000000000000E010F110F1010161911111E0067
:20436000000E1010110E01010D1311110F00000E111F100E0609081C080808000F11110FB6
:20438000010E1010161911111104000C0404040E0200060202120C101012141814240C0492
:2043A000040404040E00001A151511110000161911111100000E1111110E00001E111E106B
:2043C0001000000D130F01010000161910101000000E100E011E08081C0808090600001196
:2043E0001111130D00001111110A040000111115150A0000110A040A11000011110F010E6A
:2044000000001F0204081F03040408040403040404040404040C02020102020C00081502D6
:204420000000001F1F111F111F1F00000E0A0A0A0E0000040C04040400000C0204080E0041
:20444000000C0204020C00000A0A0E020200000E080C020C000006080E0A0E00000E02049E
:20446000080800000E0A0E0A0E00000E0A0E020C1F1F1F1F1F1F1F1F1F1F1F1F1F1F1F1FCA
:204480001F1F1F1F1F1F1F1F1F1F1F1F1F1F1F1F1F1F1F1F1F1F1F1F1F1F1F1F1F1F1F1F3C
:2044A0001F1F1F1F1F1F1F1F1F1F1F1F1F1F1F1F1F1F1F1F1F1F1F1F1F1F1F1F1F1F1F1F1C
:2044C0001F1F1F1F1F1F1F1F1F1F1F1F1F1F1F1F1F1F1F1F1F1F1F1F1F1F1F1F1F1F1F1FFC
:2044E0001F1F1F1F1F1F1F1F1F1F1F1F1F1F1F1F1F1F1F1F1F1F1F1F1F1F1F1F1F1F1F1FDC
:204500001F1F1F1F1F1F1F1F1F1F1F1F1F1F1F1F1F1F1F1F1F1F1F1F1F1F1F1F1F1F1F1FBB
:204520001F1F1F1F1F1F1F1F1F1F1F1F1F1F1F1F1F1F1F1F1F1F1F1F1F1F1F1F1F1F1F1F9B
:204540001F1F1F1F1F1F1F1F1F1F1F1F1F1F1F1F1F1F1F1F1F1F1F1F1F1F1F1F1F1F1F1F7B
:204560001F1F1F1F1F1F1F1F1F1F1F1F1F1F1F1F1F1F1F1F1F1F1F1F1F1F1F1F1F1F1F1F5B
:204580001F1F1F1F1F1F1F1F1F1F1F1F1F1F1F1F1F1F1F1F1F1F1F1F1F1F1F1F1F1F1F1F3B
:2045A0001F1F1F1F0102040000000010080400000000000A00000000000400040810110E13
:2045C0000404000404040400000D1212120D0609090E0909160000091502020200000004FD
:2045E0000A111F060804020F110E00000E101E100E06040404040406000804020609110097
:20460000001212121D1000001F0A0A0A13000609090E08101F08040204081F00000F12121E
:20462000120C00000F1404050204040E150E04040E1111110A0A1B1F00110A040A111F0005
:2046400011110F010E05020500000000000000000000150002060E060200040404000000CF
:2046600000020202040808080000001F0000000E020E080E00000E0A0E000000000C02048D
:20468000020C00000000000000000008001808080A04040A1E111E101010090A040A12010F
:2046A0001F11141C14101000000E111E100C0000040404040711191D1F171311140A05052D
:2046C000050A1400081C1E1C08001F1F1F1F1F1F1F1F1B110A1B1B1B1F1B151115151F1F0A
:2046E0001B1D1915191F0000000000001F040E150404001F040A0E0A0A001F0402060A0644
:20470000001F00000804020100181C0E070301001F0F0703010000000010181C1E1F000262
:20472000051D05020000040A0A0A040000100004000100040E1F0E0E0E00000E0E0E1F0E63
:0847400004150A150A150A15FB
:00000001FF
